:020000020000FC
:1000000008C007C006C002C004C003C012BE53959A
:100010001895F8945527442702E009BF00E1C498D9
:10002000BC9ABB98C398442705E702BF102EE1E0B5
:10003000FF2774E0F3BFBCE0C1E191E5A4EFB19B01
:10004000FECFE3BF7894B19B04C0F894A51708F3E2
:10005000F9CFF8945B17E8F2C517D8F27894B19904
:1000600004C0F894A517A8F2F9CFF894591788F2AC
:1000700012BE55274395741709F0E4CF4A95BC98F2
:06008000C49ABB9ADFCF19
:00000001FF
